:1000000012C02CC02BC02AC029C028C027C026C0BF
:1000100025C024C023C022C021C020C01FC01EC0D4
:100020001DC01CC01BC011241FBECFE5D4E0DEBF25
:10003000CDBF10E0A0E6B0E0E2E8F1E002C005903C
:100040000D92A036B107D9F710E0A0E6B0E001C0EC
:100050001D92A036B107E1F767D092C0D1CFCF9300
:10006000DF93CDB7DEB7E8E3F0E01082E5E3F0E040
:1000700080E28083E2E3F0E01082E7E3F0E01082C8
:10008000E4E3F0E080E28083E1E3F0E01082DF91DE
:10009000CF910895CF93DF93CDB7DEB723970FB6F7
:1000A000F894DEBF0FBECDBF89838981282F332707
:1000B0003B832A838A819B81009731F02A813B818F
:1000C0002130310549F010C0A5E3B0E0E5E3F0E0F0
:1000D00080818F7D8C931FC0A5E3B0E0E5E3F0E065
:1000E000808180628C9317C0E5E3F0E080819927DE
:1000F00080729070009741F0A5E3B0E0E5E3F0E096
:1001000080818F7D8C9307C0A5E3B0E0E5E3F0E04C
:10011000808180628C9323960FB6F894DEBF0FBE69
:10012000CDBFDF91CF910895CF93DF93CDB7DEB7E9
:1001300022970FB6F894DEBF0FBECDBF90DF80E0F0
:10014000A9DF80E69AEE9A83898305C089819A8126
:1001500001979A83898389819A810097B9F781E011
:1001600099DF80E69AEE9A83898305C089819A8116
:1001700001979A83898389819A810097B9F7DFCFA4
:02018000FFCFAF
:00000001FF
